:020000020000FC
:1000000085C613C0000000000000000000000000D2
:10001000000027C10BC0FFC0000001C100000000AC
:10002000ABC0000000000000000018951FB6409112
:1000300086005091870091FD29C06091810097FF53
:100040006F7B97FD6064609381009260C3B097FD01
:10005000C094C0FE03C0742E852E8AC060918100BA
:1000600097FF606497FD6F7B6093810066276062F5
:1000700066BB9D7F40E050E0C3B097FDC094C0FCDC
:100080006DC050931C0140931B0168C060918100BA
:1000900097FF606497FD6F7B609381009D7F83FF76
:1000A0003EC06091810097FF6F7B97FD6064609315
:1000B00081006627606266BB92604093190150938D
:1000C0001A0160911701B0901801461B5B09B02C12
:1000D000443B60E0560720F466276062B62E17C0E6
:1000E000483661E0560720F466276061B62E0FC0DF
:1000F000403D62E0560720F466276860B62E07C0D0
:10010000403A65E0560718F466276460B62E4091C1
:10011000190150911A014093170150931801471982
:10012000580995FD09C094FD09C05695479593FD62
:1001300005C05695479502C0440F551F4A3F5005CC
:1001400008F04AEF50911B0150931C0140931B0192
:1001500083FF04C06CE3609596239B2940E2D42E74
:10016000916083FD05C050916F005F7D50936F00DB
:1001700050E1E52E1FBE18951FB6DD2011F0DA9470
:1001800021C040E050E063B197FD609560FD4AEF0B
:100190006091810097FF606497FD6F7B60938100A1
:1001A0006627606266BB9D7F63B197FD609560FDC9
:1001B0005AEF451731F750E2D52E40931C0140937A
:1001C0001B019160EE2011F0EA9408C050916F007D
:1001D000506250936F005527506256BB90FF19C074
:1001E00050911C0140911B0195FD450F95FD4795D0
:1001F0009E7F50912A01451710F440912A01572FF4
:10020000507F552331F4242E40912801433008F0CB
:10021000422C1FBE18951FB67E7F1FBE18951FB6B5
:1002200052E040911B01415018F000921E0109C09C
:1002300040911E014F3F29F040911E01439540938C
:100240001E0160912801623011F420900D013214DA
:1002500031F010F03A9401C033945A9591F71FBED3
:1002600018951FB6601429F06092B20066241FBE74
:10027000189581FF0994452D089496FF440F10F0BE
:10028000642E40E04093B20050B78D7F652D6A3FE9
:1002900088F445B1497F45B94BB14F7D4BB982FFD9
:1002A00009C042E04A95F1F74BB14A614BB9816010
:1002B00055FF8E7F1FBE1895826042C05D982A9AB6
:1002C00082603EC029985D9A82603AC02A98299A35
:1002D000826036C04FE059985B984A95E1F75D9887
:1002E0002A9A82602DC04FE059985C984A95E1F7B0
:1002F0005D982A9A826024C04FE05C9859984A958C
:10030000E1F729985D9A82601BC04FE05C985B988A
:100310004A95E1F729985D9A826012C04FE05B9898
:100320005C984A95E1F72A98299A826009C04FE0C3
:100330005B9859984A95E1F72A98299A826000C0FB
:10034000452D4095089496FF440F10F0642E40E030
:100350004093B2001FBE18950000089521E00AC026
:1003600023E008C02AE006C02EE104C024E602C053
:1003700028EC00C014E000ECEFDF0A95E9F71A95CD
:10038000D1F72A95B9F7089535E120E509C032E1A2
:1003900024E606C03FE028E703C03CE02CE800C0AC
:1003A0005C9A06E90A95F1F70CE02A9AD5DF0A95DE
:1003B000E9F72A9810E4032FCFDF0A95E9F71A9599
:1003C000D1F72A9569F75C980895009128010330C8
:1003D00008F028C0009103011091040122E00038C8
:1003E000120770F0422C0092050100920601009263
:1003F0000701009208010092090100920E0112C04B
:10040000232D2095221F221F322F279531703395DF
:100410002E7F20543009209305013093060101E01E
:1004200000930E01089500910E010015E1F0009176
:100430000501109106012091030130910401021B76
:10044000130B2FEF0038120744F020E00F3712078C
:100450000CF405C00FE710E002C000E81FEF0093A6
:100460000A0110930B01089500910E01001581F10E
:1004700020910701309108019090090100910A0133
:1004800010910B01200F311F911E10EF91164CF0AF
:100490001FE091160CF409C02FEF3FEF1FE0912EE3
:1004A00004C020E030E010EF912E10911F014116A2
:1004B000142D18F4113020F005C000234AF002C0BA
:1004C000002332F420930701309308019092090130
:1004D000089500910E010015E9F100910A0111271C
:1004E00007FD1095000F111F3091260130FD05C04A
:1004F000343089F0159507950EC0A12E902EA59445
:100500009794090D1A1D353031F015950795333044
:1005100011F0159507952FEF0038120744F020E0F1
:100520000F3712070CF405C00FE710E002C000E817
:100530001FEF232D00233AF0201B18F0213008F084
:1005400007C021E005C00195200F08F001C02FEF82
:1005500020930C01089500910E010015D9F110911E
:100560000801209109013091270130FD05C0343088
:1005700089F0259517950EC0A22E912EA5949794DB
:10058000190D2A1D353031F025951795333011F0AE
:10059000259517950FEF1030200744F000E01F3F1E
:1005A00020070CF405C01FEF20E002C010E02FEF81
:1005B00000910C0122233AF0011B18F0013008F0E1
:1005C00008C001E006C010951395010F08F001C0A6
:1005D0000FEF402E089507EC00937C0000917A0005
:1005E0000068006400937A0020917A0026FDF3CF22
:1005F000009178001091790020917A002F77209354
:100600007A0024EB2093210121E02093220121E0B4
:100610002093200124EB31E0220F331F0217130730
:10062000C8F0209321013093220122E02093200181
:1006300024EB31E0922EA32E220F331F290D3A1DF9
:100640000217130738F0209321013093220123E091
:1006500020932001089507EC00937C0000917A001C
:100660000068006400937A00089520917A0026FDC6
:10067000FCCF009178001091790020917A002F77BB
:1006800020937A000F3F23E0120778F42091210194
:10069000309122010217130740F400911F0100233B
:1006A00059F00A9500931F0107C000911F010F3FE9
:1006B00019F0039500931F01401608F4042D502EE5
:1006C000089574FD02E375FD00E576FD00E577FD14
:1006D00008E2172F107F112399F020912B0123306E
:1006E00061F0102F169520FD01C0169522FD02C065
:1006F000011B03C0010F08F40FEF202E402E502ED7
:100700000895C8EBDBE0C0931501D09316012FEFDD
:100710003FE1209313013093140120930F01309394
:1007200010013695279520931101309312011FEF88
:10073000109304010FEF009303010895C091150178
:10074000D091160104C0C0910F01D0911001F8940E
:100750000091840010918500C00FD11FD0938900B3
:10076000C09388007894716020910101309102015A
:100770000093010110930201021B130B209103014E
:1007800030910401E901D695C795D695C7952C1BE4
:100790003D0B200F311F209303013093040108F01B
:1007A00008951FEF109304010FEF009303010895C4
:1007B00070FDFECFC0911101D0911201F89400910B
:1007C0008400109185000C0F1D1F10938900009369
:1007D00088007894716008950091030110910401DC
:1007E00016950795169507951695079516950795ED
:1007F0000550100918F00530100510F405E0112718
:10080000009313011093140100930F011093100132
:10081000169507950093110110931201089570FD2C
:10082000FECFC0910301D0910401F894009184009F
:10083000109185000C0F1D1F1093890000938800F4
:10084000789471600895789470FF089582FD01C0D6
:1008500004C080FDF8CF7894089506E0252D2095FA
:100860002295269527702395F8940A95F1F710B7ED
:1008700015FDE9CF2A95D9F778940895789470FFFB
:10088000089582FD01C004C080FFF8CF78940895D8
:1008900006E0252D20952295269527702395F8941E
:1008A0000A95F1F710B715FFE9CF2A95D9F7789493
:1008B0000895C0911301D0911401F894009184001F
:1008C000109185000C0F1D1F109389000093880064
:1008D00078947160089570FDFECF0895F894AEE8A5
:1008E000B1E0FD015C98599A00917B000F7B009369
:1008F0007B0078940895F894A5E8B1E0FD0129986B
:1009000081FD5D9A00917B00006400937B0003E011
:1009100000937C0078940895F894ACE7B1E0FD0171
:1009200059985B9A00917B00006400937B0002E081
:1009300000937C0078940895F894A3E7B1E0FD015A
:100940005D9881FD2A9A00917B000F7B00937B00CC
:1009500078940895F894AAE6B1E0FD015B985C9A5A
:1009600000917B00006400937B0003E000937C0017
:1009700078940895F894A7E9B1E0FD012A9881FDE3
:10098000299A00917B00006400937B0002E00093B1
:100990007C0078940895F8945C98599A00917B00B3
:1009A0000F7B00937B0078940895F894A2E6B1E061
:1009B000FD01299881FD5D9A00917B000064009300
:1009C0007B0003E000937C0078940895F894599894
:1009D0005B9A00917B00006400937B0002E000932F
:1009E0007C0078940895F894AEE5B1E0FD015D983F
:1009F00081FD2A9A00917B000F7B00937B00789405
:100A00000895F8945B985C9A00917B0000640093D1
:100A10007B0003E000937C0078940895F894A6E6A8
:100A2000B1E0FD012A9881FD299A00917B000064C4
:100A300000937B0002E000937C0078940895ACE57D
:100A4000B1E0FD0105B1097F05B90BB10F7D0BB90F
:100A50000BB1057E0BB90895009115011091160197
:100A6000083E23E0120708F4089500911501109143
:100A700016010550104000931501109316010895BA
:100A800070FDFECF089504E00093260104E000937A
:100A9000270101E00093280103E000932B019064FB
:100AA0009F770895F999FECF11BD22BDF89A00B540
:100AB0000895F999FECF00BD11BD22BDF894FA9AB0
:100AC000F99A7894089518E020E00FEFF2DF19E02A
:100AD00020E00FEFEEDF089518E020E005EAE9DFFF
:100AE00019E020E00AE5E5DF089518E020E0DADF0C
:100AF000053A31F519E020E0D5DF0A3509F510E0B7
:100B000020E0D0DF0093260111E020E0CBDF00934E
:100B1000270112E020E0C6DF0093280115E020E065
:100B2000C1DF00932B0116E020E0BCDF906401FDE3
:100B30009F7B17E020E0B6DF9F7701FD906802C041
:100B4000A2DF01D00895BFDF01E0009323010091EF
:100B50002601009324012CD002E000932301009190
:100B600027010093240124D003E000932301009186
:100B70002801009324011CD004E00093230100917C
:100B80002B010093240114D005E00093230101E020
:100B900096FF02E0009324010BD006E000932301AE
:100BA00001E097FD02E00093240102D095DF089553
:100BB0003091230100912401313051F0323061F045
:100BC000333071F0343081F0353091F03630A1F0AF
:100BD00010E020E06EDF14C011E020E06ADF10C0FA
:100BE00012E020E066DF0CC015E020E062DF08C004
:100BF00016E020E05EDF04C017E020E05ADF00C00E
:100C0000089505E0902EB4DB9A94E9F70895F894DE
:100C1000BBDBBDDBBFDBC1DBA5DBB6DBB8DBBADB37
:100C2000BCDBA0DBB1DBB3DBB5DBB7DB78940895CD
:100C300090902301A0902401F894A6DBA5DBA4DB0F
:100C400091DB9A94D1F7A9DB8DDBAA94E1F7789434
:100C50000895F894A2DB789489DB00911B010130A0
:100C6000C0F7F89491DB7EDB8FDB78947FDB00911B
:100C70001B010A3FB0F3CBDFC4DFC3DF01E0009309
:100C8000230101E00093240100E000932501D0DF5F
:100C900005E0902E6DDB00911B01013040F413DF65
:100CA00087DF1ADFB4DF08E000936000AADF9A94C0
:100CB00089F700912501039500932501033008F47D
:100CC000E6CF9FDF0091240103950093240115E0F6
:100CD00000912301033009F413E000912301053052
:100CE00008F012E0139500912401011708F4CCCF0D
:100CF00088DF87DF009123010395009323010730EC
:100D000008F4BFCF08E0009360007BDFF894A8955B
:100D100004B7007004BF0091600008610093600098
:100D200000E00093600000E80093610001E00093A0
:100D3000610004E00EBF0FEF0DBF81DE00E005B9DA
:100D400006E104B900E008B900E007B900E00BB91A
:100D50000AE30AB90024A0E0B0E00D92AA31E9F755
:100D6000A0E0B1E004E60D920A95E9F768DE02E042
:100D700005BD02E00093810001E00093B10083DE35
:100D8000B4DEF6DA01DBF0DA02DBEEDA03DBECDA12
:100D900001E005BB00936E0003E006BB00936F000B
:100DA00001E007BB0093700000917A0002600160CF
:100DB00000937A0078940FDC0091810097FF006423
:100DC00097FD0F7B0093810000916F0000620093FC
:100DD0006F000027006206BB9D7FCADAC1DA00916E
:100DE0001B010130D8F7C4DA886015E0912EB8DA1B
:100DF00090FFFECF00911B010230B8F3292F2C7316
:100E000030911D0120931D01231779F79A9479F7EA
:100E1000877F0091810097FF006497FD0F7B00930F
:100E200081000027006206BB9D7FF894ADDAACDA42
:100E3000ABDA78949DDA00920D0192DA00911B01F1
:100E40000A3F08F006CF10910D01011710F0009332
:100E50000D01013090F7F894A0DA9FDA9EDA7894C9
:100E600087DA7EDA00911B010130D8F3E8DD222415
:100E70003324442455240FEF00931F0100920501F1
:100E800000920601009207010092080100920901F8
:100E900000920E017727882700921E0100917A00A8
:100EA0000F7700937A0000917B00006400937B0031
:100EB00028DC8460706105DC5DDD50DA0FDD4EDA20
:100EC0004DDA19DD4DDA28DD4BDA4ADA35DD4ADA5A
:100ED00041DD46DA43DA7F7E7062F3DB4BDD2EDCE8
:100EE0007BDCBADDCDDDFADC29DC76DCB5DDC8DD06
:100EF00002DD24DC71DCB0DDC3DD0EDD1FDC6CDC6B
:100F0000ABDDBEDD19DD1ADC67DCA6DDB9DD22DD77
:100F100015DC62DCA1DD0091150110911601083E7F
:100F200023E0120710F0ACDDD9CF7F7D7064C9DB00
:100F300002E000930001A4DD1DDD00DC4DDC8CDD52
:100F40009FDDCCDCFBDB48DC87DD9ADDD4DCF6DB27
:100F500043DC82DD95DDE0DCF1DB3EDC7DDD90DD38
:100F6000EBDCECDB39DC78DD8BDDF4DCE7DB34DC7F
:100F700073DD009100010A9521F00093000180DDEE
:100F8000DBCF7F7B70689DDB7BDDF4DCDCDB10DCA2
:100F900023DC45DC01E00093000155DC70FF97C0C5
:100FA00088DC99DC9BDCCFDB03DC16DC38DC66DC20
:100FB00070FF8DC07EDC8FDC9EDCC5DBF9DB0CDCDA
:100FC0002EDC41DC70FF83C074DC85DCA5DCBBDB80
:100FD000EFDB02DC24DC52DC70FF79C06ADC7BDCF6
:100FE000ABDCB1DBE5DBF8DB1ADC2DDC70FF6FC0BE
:100FF00060DC71DCAFDCA7DBDBDBEEDB10DC3EDCD6
:1010000070FF65C056DC67DCB5DC9DDBD1DBE4DB63
:1010100006DC009100010A9519F000930001BDCF94
:10102000F8948B7F0BB1057E0BB95C9AA6E6B1E014
:10103000FD01789408DC70FF4AC03BDCC6D94BDC6C
:10104000AADC81DBB5DBC8DBEADB18DC70FF3FC064
:1010500030DCE9D940DCA9DC76DBAADBBDDBDFDBF9
:10106000F2DB70FF34C025DCFFD935DCAFDC6BDB95
:101070009FDBB2DBD4DB02DC70FF29C01ADC29DA8B
:101080002ADCB1DC60DB94DBA7DBC9DBDCDB70FFD7
:101090001EC00FDC60DA1FDCB4DC55DB89DB9CDBB7
:1010A000BEDBECDBD8DA70FF12C003DCDEDA13DC67
:1010B000B5DC49DB7DDB90DBB2DB7F7700911E0185
:1010C000013028F40091040107FD09F4B3CFB7DC27
:0A10D000222433244424552488CE42
:00000001FF
